S02100002E2E5C62696E5C64656D6F70726F675F73746D3332663039312E7372656341
S3150800200000800020F52C0008472D0008492D0008FF
S3150800201000000000000000000000000000000000B2
S315080020200000000000000000000000004B2D000822
S3150800203000000000000000004D2D0008012E0008D9
S31508002040532D0008552D0008572D0008592D000856
S315080020505B2D00085D2D00085F2D0008612D000826
S31508002060632D0008652D0008672D0008692D0008F6
S315080020706B2D00086D2D00086F2D0008712D0008C6
S31508002080732D0008752D0008772D0008792D000896
S315080020907B2D00087D2D00087F2D0008812D000866
S315080020A0832D0008852D0008872D0008892D000836
S315080020B08B2D00088D2D00088F2D0008912D000806
S315080020C0EE11AA5510B5064C2378002B07D1054BFF
S315080020D0002B02D0044800E000BF0123237010BD86
S315080020E03C010020000000000C300008084B10B529
S315080020F0002B03D00749084800E000BF07480368DB
S31508002100002B00D110BD064B002BFBD09847F9E7F2
S3150800211000000000400100200C3000083C010020AF
S3150800212000000000164B002B00D1144B9D464022A0
S3150800213092029A1A924600218B460F461348144A71
S31508002140121A00F036FF0F4B002B00D098470E4BA3
S31508002150002B00D098470020002104000D000D48F0
S31508002160002802D00C4800E000BF00F0F3FE200073
S31508002170290000F0B5FD00F0D7FEC04600000800B3
S315080021800080002000000000000000003C01002044
S31508002190AC010020000000000000000070B588B007
S315080021A08024A4020121200000F090FC01212000D7
S315080021B000F07EFC9025ED0501220221280000F0A2
S315080021C06DFB01220321280000F068FB06A90C26F6
S315080021D0069603234B71013B0B7100248C71013B5E
S315080021E0CB71280000F014FBE1231B020093019435
S315080021F00294039405940496054C6946200000F061
S3150800220081FC0121200000F0EBFC08B070BDC0463F
S3150800221000440040F0B557464E46C0B48DB08146DE
S315080022208A46019202A800F04BFB049B0093002506
S3150800223021E0154A6B009E5CD3185F78F4190134C7
S315080022404B465C432100009800F068FE002910D137
S315080022502100009800F0DCFD80B253461880013852
S3150800226080B20A4B984204D8019B1E705F70012009
S3150800227004E00135EDB2112DDBD900200DB00CBC00
S3150800228091469A46F0BDC046E02F0008FF030000BD
S31508002290F0B58BB06B469E1C0123338002222C4975
S315080022A0684600F07DFE01218020800400F00EFCC7
S315080022B001218020C00200F0FBFB264D04220821E4
S315080022C0280000F0EBFA04220921280000F0E6FABB
S315080022D008A9C0239B00089302230B7101334B7195
S315080022E000248C7101270123CB71280000F090FA95
S315080022F06A4631001848FFF78DFF184800F00EF9B6
S3150800230005AD280000F018FAAC71EC712C726C72ED
S31508002310AC72EC72AC70EC706B461B78013B2B719F
S315080023206B465B78013B6B7133882B8029000B4821
S3150800233000F000F901A88472C4720773048044800F
S315080023408480C4800481477300F078F90BB0F0BD2F
S31508002350DC2F00080004004820A1070000640040A4
S3150800236010B504002021064800F04AFC012805D1D2
S31508002370034800F041FC2070012000E0002010BD59
S315080023800044004010B5FFF709FFFFF781FF10BDB5
S31508002390BFF34F8F024A034BDA60BFF34F8FFEE756
S315080023A00400FA0500ED00E010B5214B1B78002B60
S315080023B013D12048FFF7D4FF012837D11D4B1B78CE
S315080023C0002B33D000F016FD1B4B18600122184B6A
S315080023D01A700022194B1A7028E0184B1878013029
S315080023E0144B1818FFF7BCFF012815D1134A1378A8
S315080023F00133DBB213700F4A1278934216D10022CA
S315080024000B4B1A700B4B5B78FF2B0FD1094B9B7844
S31508002410002B0BD1FFF7BCFF00F0ECFC064B1B684A
S315080024206433984202D90022014B1A7010BDC04687
S315080024309A010020580100209C01002099010020E3
S3150800244000B587B000210D4800F0D4F9002812D055
S3150800245001AA0021094800F07FF9094B019A9A421E
S3150800246009D101ABDB7AFF2B05D101AB1B7B002B16
S3150800247001D1FFF78DFF07B000BDC04600640040DC
S315080024806706000010B5FFF78FFFFFF7D9FF10BDED
S3150800249010B582B001218020800200F009FB2023BC
S315080024A000931F3B6A461371002393710322694602
S315080024B04A71CB719024E405200000F0A9F9202187
S315080024C0200000F0E9F902B010BDC04610B500F0D2
S315080024D091FC04000F4B1B68C31AF422FF32934287
S315080024E017D90D4B1B78002B09D1F33AFF3A0A4B43
S315080024F01A7020219020C00500F0CCF907E00022D0
S31508002500054B1A7020219020C00500F0C5F9014B33
S315080025101C6010BDA0010020A401002010B5802475
S31508002520A4040121200000F0DFFA0021200000F0B9
S31508002530DBFA10BD10B503680222934303600268F4
S31508002540012313430360002300E001334268D207E6
S3150800255002D4394A9342F8D14368DB0768D58B79A8
S31508002560012B04D102687F331343036003E0036839
S31508002570802293430360CB79012B04D102683F3351
S315080025801343036003E003684022934303600B7A16
S31508002590012B04D102681F331343036003E0036869
S315080025A02022934303604B7A012B04D102680F3330
S315080025B01343036003E003681022934303608B7A96
S315080025C0012B04D1026807331343036003E0036851
S315080025D0082293430360CB7A012B04D102680333A4
S315080025E01343036003E003680422934303608B7874
S315080025F09C07CA78130623430A79120413434A79B7
S31508002600120513430A88013A1343C361036801227A
S3150800261093430360002300E001334268D20702D5E2
S31508002620054A9342F8D14368DB0703D5002002E048
S31508002630002000E0012010BDFFFFFF0070B5837A7F
S31508002640012214009C403B4B802189005D582A4397
S315080026505A508725AD005959E24311405951037B19
S31508002660002B17D13349103D4B5913404B51837AF0
S31508002670C5882D04468835434833DB005D50837A88
S3150800268081880904058829434833DB00294DAC466F
S3150800269063445960037B012B18D126498325AD0075
S315080026A04B5923434B51837A05882D044688354375
S315080026B04833DB005D50837A81880904C58829433D
S315080026C04833DB001B4DAC4663445960C37A002B84
S315080026D006D1184D812189006B5813406B5005E0CF
S315080026E0144D812189006B5823436B500389002BB5
S315080026F005D1104985239B00CD582A40CA50038925
S31508002700012B05D10B49852292008B5823438B5008
S31508002710437B012B05D10749872292008B581C431E
S315080027208C500449802292008B58012083438B5099
S3150800273070BDC0460064004000238371C3710372F4
S3150800274043728372C3728370C37003330371013B90
S315080027504371013B0380704730B50B001B331B01E7
S315080027601B5804242340137206D10B001B331B018C
S315080027701B585B0D136005E00B001B331B011B5830
S31508002780DB0853600B001B331B011C5802252C4029
S315080027905472C3185C680D352C4094725B681B0A2A
S315080027A0D3740B01C3181C00B934FF342568D572DD
S315080027B025682D0A157325682D0C55732468240E73
S315080027C09473BD33FF331C68D4731C68240A1474CD
S315080027D01C68240C54741B681B0E9374002904D1BE
S315080027E0C26820231343C36003E00269202313430E
S315080027F0036130BD002903D1C0680323184006E0F1
S31508002800012903D100690323184000E0002070471E
S3150800281070B500223AE0012393400C681C40A3429D
S3150800282033D10B79013BDBB2012B17D883685500EE
S315080028300324AC40A343836084684B79AB402343AD
S31508002840836083881404240C0125A540AB43838048
S3150800285085888B79A3402B439BB2838003685500F8
S3150800286003242600AE40B343036006680B79AB40E9
S3150800287033430360C3681604F60BB440A343C3602E
S31508002880C468CB79AB402343C36001320F2AC2D94F
S3150800289070BDC046816170470185704730B5072312
S315080028A00B409B009A40C908083189000C580F252F
S315080028B09D40AC430C500B581A430A5030BDC046D5
S315080028C0F8B50400734B5B680C221340042B0CD03C
S315080028D002D8002B05D029E0082B0AD00C2B21D0D2
S315080028E024E06D4B0360002023E06B4B036000205F
S315080028F01FE0684B58685A68C0235B02800C0F2596
S315080029002840851C1A4202D16448684308E0614B96
S31508002910DB6A0F21194001315F4800F079FA6843F4
S31508002920206006E05E4B0360002002E05A4B2360FD
S31508002930002058494B681B090F221340594DEB5C80
S31508002940DBB226683200DA40130062604A68120A6F
S3150800295007273A40AA5CD2B2D340A3600A6BD205D5
S3150800296002D4514AE26008E04A4A5268520402D444
S315080029705A08E26001E09A08E260464A126B52067B
S3150800298002D44A4A226102E0802212022261414AA6
S31508002990126BD20602D4404A626100E066613D4A83
S315080029A0126B920701D1A36119E03A4A126B03210F
S315080029B00A40012A01D1A66111E0364A126B0321A9
S315080029C00A40022A03D180221202A26107E0314A94
S315080029D0126B03210A40032A01D12F4AA2612D4A0C
S315080029E0116BC0229202114201D1E36120E0294A0B
S315080029F0116BC02292020A40802149028A4201D103
S31508002A00E66115E0234A116BC02292020A40802132
S31508002A1089028A4203D180221202E26108E01D4A35
S31508002A20126BC02189020A408A4201D11A4AE26120
S31508002A30184A116BC0221203114201D1236220E009
S31508002A40144B1A6BC0231B0313408022D2029342F5
S31508002A5001D1266215E00F4B1A6BC0231B031340E6
S31508002A6080221203934203D180231B02236208E0CB
S31508002A70084B1B6BC02212031340934201D1064B2D
S31508002A802362044B1B6B1B0602D4054B636200E0F2
S31508002A906062F8BD0010024000127A0000093D008D
S31508002AA0006CDC02C0000020809FD5001280000068
S31508002AB0002904D0044B5A691043586103E0024ABE
S31508002AC0536983435361704700100240002904D0BC
S31508002AD0044BDA691043D86103E0024AD369834399
S31508002AE0D361704700100240002904D0044B1A69CC
S31508002AF01043186103E0024A136983431361704760
S31508002B0000100240F0B58DB004000D0003680122E4
S31508002B109343036042682B4B13408A681343436010
S31508002B200168294B19406B68EA6813432A691A43F6
S31508002B300B00134303608268244B13406A691343EE
S31508002B40836002A8FFF7BCFE214B9C4201D1089E78
S31508002B500AE0204B9C4201D1099E05E01E4B9C428F
S31508002B6001D10A9E00E0049E23681B040CD576005A
S31508002B702B6801931900300000F04AF90700019903
S31508002B80300000F0CBF90AE02B68019319003000F9
S31508002B9000F03EF907000199300000F0BFF92B68F4
S31508002BA05B08994200D3013723681B0406D57B08C6
S31508002BB007221A40094B3B401A431700BBB2A381B0
S31508002BC00DB0F0BDFFCFFFFFF3E9FFFFFFFCFFFFEE
S31508002BD0003801400044004000480040F0FF000073
S31508002BE0002904D0026801231343036003E0036845
S31508002BF00122934303607047808CC005C00D70475F
S31508002C00C369194201D0012000E000207047C04680
S31508002C101122144B1A60144B5A685A605A685A6043
S31508002C205968124A0A405A605A68A02189030A4319
S31508002C305A601A68802149040A431A600A4B1B68BD
S31508002C409B01FBD5084B5A6803218A435A60596889
S31508002C5002220A435A60044B5B680C221340082B75
S31508002C60F9D170470020024000100240FF7FC0FFE4
S31508002C7010B5124B1A6801210A431A605868104A9F
S31508002C8002405A6018680F4A02401A6018680E4ACD
S31508002C9002401A6058680D4A02405A60DA6A0F20E4
S31508002CA08243DA62186B0A4A02401A635A6B8A43ED
S31508002CB05A6300229A60FFF7ABFF10BD001002406E
S31508002CC00CB8FFF8FFFFF6FEFFFFFBFFFFFFC0FF94
S31508002CD0ACFEFFFF10B5FFF7DBFB00F065F810BD93
S31508002CE010B5FFF7F7FFFFF74DFBFFF7EFFBFFF711
S31508002CF0C9FBFAE708498D460849094A094B9B1A50
S31508002D0005DD00240859105104349C42FADB0648B4
S31508002D108047064800470000008000201830000859
S31508002D20C00000203C010020712C00082521000865
S31508002D301849194A002301E00B6004319142FBD37C
S31508002D40FFF7CEFFFEE7FEE7FEE7FEE7FEE7FEE754
S31508002D50FEE7FEE7FEE7FEE7FEE7FEE7FEE7FEE73D
S31508002D60FEE7FEE7FEE7FEE7FEE7FEE7FEE7FEE72D
S31508002D70FEE7FEE7FEE7FEE7FEE7FEE7FEE7FEE71D
S31508002D80FEE7FEE7FEE7FEE7FEE7FEE7FEE7FEE70D
S31508002D90FEE7FEE73C010020AC010020014B18606D
S31508002DA07047C046A801002010B50E4B1868FA21D6
S31508002DB0890000F02DF801380B4B98420DD80B4AC4
S31508002DC050600B490B6A1B021B0AC020000603430E
S31508002DD00B6200239360073313600020FFF7DEFFC2
S31508002DE010BDC046D0000020FFFFFF0010E000E045
S31508002DF000ED00E0014B18687047C046A8010020A6
S31508002E00024A1368013313607047C046A8010020C0
S31508002E10002243088B4274D303098B425FD3030A0B
S31508002E208B4244D3030B8B4228D3030C8B420DD31E
S31508002E30FF22090212BA030C8B4202D312120902AC
S31508002E4065D0030B8B4219D300E0090AC30B8B42EA
S31508002E5001D3CB03C01A5241830B8B4201D38B0398
S31508002E60C01A5241430B8B4201D34B03C01A52413D
S31508002E70030B8B4201D30B03C01A5241C30A8B4280
S31508002E8001D3CB02C01A5241830A8B4201D38B026B
S31508002E90C01A5241430A8B4201D34B02C01A52410F
S31508002EA0030A8B4201D30B02C01A5241CDD2C30981
S31508002EB08B4201D3CB01C01A524183098B4201D3FD
S31508002EC08B01C01A524143098B4201D34B01C01AE8
S31508002ED0524103098B4201D30B01C01A5241C30860
S31508002EE08B4201D3CB00C01A524183088B4201D3CF
S31508002EF08B00C01A524143088B4201D34B00C01ABB
S31508002F005241411A00D20146524110467047FFE726
S31508002F1001B5002000F006F802BDC0460029F7D02A
S31508002F2076E770477047C046084B10B50400002B7B
S31508002F3002D0002100E000BF054B1868836A002B09
S31508002F4000D09847200000F03CF8C046000000007A
S31508002F50083000080E4B70B500251E000D4CE41A0B
S31508002F60A410A54204D0AB00F35898470135F8E7FA
S31508002F7000F028F8084B00251E00084CE41AA41097
S31508002F80A54204D0AB00F35898470135F8E770BD61
S31508002F9034010020340100203401002038010020CB
S31508002FA0002310B59A4203D0CC5CC4540133F9E728
S31508002FB010BD03008218934202D019700133FAE754
S31508002FC07047FEE7F8B5C046F8BC08BC9E46704791
S31508002FD0F8B5C046F8BC08BC9E467047010100001B
S31508002FE005020602060307030803090309040A047F
S31508002FF00B040C040C050D050E050F050F0610062F
S315080030001007100843000000D4000020000000004C
S30D0800301014F1FF7F0100000026
S315080030180000000001020304010203040607080968
S31508003028006CDC0200000000000000000000000040
S31508003038000000000000000000000000000000007A
S31508003048000000000430000800000000000000002E
S31508003058000000000000000000000000000000005A
S31508003068000000000000000000000000000000004A
S31508003078000000000000000000000000000000003A
S3110800308800000000ED200008C52000082C
S70508002000D2
